:1000000012C0189518951895189518951895189563
:100010001895189518951895189518951895189578
:100020001895189518958FED8DBFC0ECE8EB4E2E06
:10003000DD275D2EEEE7F0E0A0E6B0E088278D93A7
:100040003197E9F766248FEF87BB8FED81BB8FEF88
:1000500088BB8FEF82BB0027A0E38C9185FB0EF459
:1000600001E041E0041709F0FCC081E080936000EA
:1000700000916000033010F009F010C086E9809311
:10008000660088E080936500E4EBF2E048D1ECD0B4
:10009000A0E68C918F5F8C9308F4EACF81E0809387
:1000A000600000916000023010F009F010C084E69A
:1000B0008093660088E080936500E4ECF2E02FD145
:1000C000D3D0A0E68C918F5F8C9308F4EACF81E0C7
:1000D0008093600000916000033010F009F010C0C0
:1000E0008AEF8093660088E080936500E4EDF2E09B
:1000F00016D1BAD0A0E68C918F5F8C9308F4EACF2A
:100100008FEB82BB86E990E019D181E0809360009B
:1001100000916000033010F009F010C084E6809375
:10012000660088E080936500E4EEF2E0F8D09CD0B1
:10013000A0E68C918F5F8C9308F4EACF81E08093E6
:10014000600000916000013010F009F010C088ECF0
:100150008093660088E080936500E4EFF2E0DFD0F2
:1001600083D0A0E68C918F5F8C9308F4EACF81E076
:100170008093600000916000013010F009F010C021
:1001800088EC8093660087E080936500E4E0F3E00C
:10019000C6D06AD0A0E68C918F5F8C9308F4EACF2A
:1001A00081E08093600000916000013010F009F060
:1001B00010C088EC8093660086E080936500E2E1E1
:1001C000F3E0ADD051D0A0E68C918F5F8C9308F412
:1001D000EACF8FEF88BB8FEF82BB88EC90E0AED088
:1001E00080E08093650080E08093670084E68093E0
:1001F000630081E08093600000916000013210F0A4
:1002000009F02AC0A7E68C918D5F8C93009167005E
:1002100043E0A7D0A6E64C9380E088BB80E482BB95
:10022000A7E68C9199278AD0A3E68C9183508C9372
:100230000091630043E0A1D0A5E60C938FEF88BB4B
:100240008FEF82BBA5E68C91992778D0A0E68C91A0
:100250008F5F8C9308F4D0CF8FEB82BB80E590E06A
:100260006DD0F5CEF894FFCF81E08093610040918E
:10027000650000916100041710F009F01AC052D017
:10028000A2E66BD00C924BD04DD0A4E666D00C9277
:1002900046D0A2E68C9188BBA4E68C9182BBA6E6F0
:1002A0008C9199274BD0A1E68C918F5F8C9308F4A9
:1002B000DECF089577FFBBFFDDFFEEBF77FFBBFF0B
:1002C000DDFFEEBF3FFE9FFDCFFDE7FBF3FBF9F740
:1002D000FCF77EFEFFBFFFF000FF00FFFFBFFFF057
:1002E00000FF00FF7FFF7BFB5BFB5AF31A73127268
:1002F00010720070DFBF9FFF1FFF1EFF1CBF18FFA3
:1003000010FF00FF10BF18FF1CFF1EFF1FBF9FFF45
:10031000DFFFFFBFFFFDFFFCFFF4FFF0FFBF8E2EEE
:100320009F2E0895E82DF92D08953197F1F708953E
:10033000689462F80895E89462F80895EF93FF9343
:10034000EE27E82BE92B31F0EAEFF0E03197F1F7F7
:100350000197D1F7FF91EF910895C895319600204C
:100360000895FF935527F8E0469508F4500F5795E8
:100370004795FA95D1F7FF910895FF93881BF9E00F
:10038000001FFA9511F4FF910895881F841B18F43B
:0A039000840F8894F5CF0894F3CF92
:00000001FF
